:020000020000FC
:1000000043C0189518951895189518950DC0189512
:10001000189538C01895189518951895189518952D
:1000200018951895189518952FB740E04DBD4CBD03
:1000300012976FEFA215B30508F06E7FA415B505F2
:1000400008F06D7FA615B70508F06B7FA815B905F8
:1000500008F0677FAA15BB0508F06F7EAC15BD05DB
:1000600008F06F7D65BBA03021F4B03011F4B7E02B
:10007000AFEF51E040E05A174B0711F4B7E0AEEF95
:100080002FBF18957727189504E00EBF0FE50DBF19
:100090000FEF04BB00E005BB08EF07BB07E008BBA0
:1000A0000FE101BB00EE02BB00E0202E302E402EFF
:1000B000502E602E702E802E902EA02EB02EC02E90
:1000C000D02E07E109B900E00BB9549A06E800BD4B
:1000D000772700E00EBB0FBB04E003BF00E00FBDBD
:1000E0000BBD06E40ABD01E00EBD01E109BFB7E0AA
:1000F000AEEF78945F9BFECF0BD1FCCF00000000E9
:1001000000000000000000000000000000000000EF
:1001100001000100010001000100020002000200D4
:1001200003000300040004000400050006000600AC
:1001300007000700080009000A000B000B000C0074
:100140000D000E000F001000120013001400150027
:100150001700180019001B001C001E001F002100C2
:1001600023002500260028002A002C002E00300045
:1001700033003500370039003C003E0041004300A9
:10018000460048004B004E005100540057005A00F2
:100190005D006000630067006A006D00710074001C
:1001A00078007C007F00830087008B008F00930025
:1001B00097009C00A000A400A900AD00B200B70009
:1001C000BB00C000C500CA00CF00D400D900DF00CA
:1001D000E400E900EF00F500FA00000106010C015F
:1001E000120118011E0124012A01310137013D01CC
:1001F00044014B01520158015F0166016D01750117
:100200007C0183018B0192019A01A101A901B10135
:10021000B901C101C901D101DA01E201EB01F30128
:10022000FC0104020D0216021F02280232023B02E8
:1002300044024E02570261026B0274027E0288027F
:1002400092029D02A702B102BC02C602D102DC02E8
:10025000E702F202FD02080313031F032A03360319
:1002600041034D035903650371037D03890396031D
:10027000A203AF03BB03C803D503E203EF03FC03F0
:10028000090417042404320440044D045B04690487
:10029000770485049404A204B104BF04CE04DD04F1
:1002A000EC04FB040A05190529053805480557051E
:1002B0006705770587059705A805B805C805D90519
:1002C000EA05FA050B061C062E063F0650066206D6
:1002D000730685069706A906BB06CD06DF06F2065D
:1002E0000407170729073C074F07620775078907A7
:1002F0009C07B007C307D707EB07FF07ECEFF0E059
:1003000080E0110F881FE10FF81F959184911895D7
:1003100000E002BF1CB000E0071751F001E0071732
:1003200059F002E0071761F003E0071769F012C007
:100330000FEF101671F00BC000E0101651F007C05F
:1003400000E0101631F003C00FE0101611F070E05D
:10035000F3C0EDC0C6B3D0B3D695D695D695D69595
:10036000D695C770D770C73019F4E09ACDB3C7706F
:10037000D73031F4E09ADDB3D695D695D695D770BF
:1003800004E0071759F4112DB9DFC03011F4292EFC
:10039000382ED030F9F4892E982EC9C005E0071701
:1003A00059F4112DABDFC03011F4492E582ED03046
:1003B00089F4A92EB82EBBC006E0071761F4112DF1
:1003C0009DDFC03011F4692E782ED03019F4C92E7B
:1003D000D82EADC0ACC007E0071759F4112D8EDF41
:1003E000C13011F4292E382ED130F9F4892E982EEF
:1003F0009EC008E0071759F4112D80DFC13011F4B9
:10040000492E582ED13089F4A92EB82E90C009E07B
:10041000071761F4112D72DFC13011F4692E782EA7
:10042000D13019F4C92ED82E82C081C00AE0071736
:1004300059F4112D63DFC23011F4292E382ED23039
:10044000A1F7892E982E73C00BE0071759F4112DD0
:1004500055DFC23011F4492E582ED23031F7A92E73
:10046000B82E65C00CE0071759F4112D47DFC230D4
:1004700011F4692E782ED230C1F6C92ED82E57C06D
:100480000DE0071759F4112D39DFC33011F4292E6F
:10049000382ED330F9F4892E982E49C00EE0071774
:1004A00059F4112D2BDFC33011F4492E582ED330BF
:1004B00089F4A92EB82E3BC00FE0071761F4112D67
:1004C0001DDFC33011F4692E782ED33019F4C92EF4
:1004D000D82E2DC02CC000E1071759F4112D0EDFC6
:1004E000C43011F4292E382ED430A1F7892E982E3D
:1004F0001EC001E1071759F4112D00DFC43011F4BB
:10050000492E582ED43031F7A92EB82E10C002E152
:10051000071759F4112DF2DEC43011F4692E782E2C
:10052000D430C1F6C92ED82E02C011CF10CF73958A
:0A05300003E1701709F40BCF0895E2
:00000001FF
